:200000001EC15DC63EC1F8CB3CC13BC1F7C4F6C438C137C136C12ECC01CC33C132C131C126
:2000200030C12FC12EC10200080012001F003100470060007E009F00C500EE001B014D01A3
:200040008201BB01F80139027E02C70213036403B90311046E04CE0433059B0507067706F0
:20006000EC066407E0076008E4086B09F709870A1A0BB20B4E0CED0C900D380EE30E920F39
:200080004510FC10B711761239130014CB1499156C1643171D18FC18DE19C41AAF1B9D1C45
:2000A0008F1D851E7F1F7D207F2184228E239C24AE25C326DD27FA281B2A412B6A2C972D12
:2000C000C82EFD2F36317332B433F93442368E37DF38333A8C3BE83C493EAD3F15418142A6
:2000E000F1436545DD465948D9495D4BE54C704E005094512B53C65466560958B0595B5BFC
:200100000B5DBE5E75602F62EE63B16578674269116BE46CBA6E9470737255743B76257810
:20012000137A067CFB7DF57FF381F583FB850488128A238C398E529070929194B696DF98EE
:200140000C9B3D9D729FABA1E8A329A66DA8B6AA03AD53AFA8B100B45CB6BDB821BB89BD8A
:20016000F5BF65C2D9C451C7CDC94CCCD0CE58D1E3D373D606D99EDB39DED8E07BE322E6EE
:20018000CEE87DEB2FEEE6F0A1F360F623F9E901B4048207550A2B0D0510E412C615AC18DC
:2001A000961B841E76216C246527632A652D6A30743382369339A83CC23FDF42004625499B
:2001C0004E4C7B4FAC52E1551A59565C975FDC6224667169C16C15706E73CA762A7A8E7D48
:2001E000F6806284D287468BBE8E3992B9953D99C49C50A0DFA372A70AABA5AE44B2E7B5B9
:200200008EB939BDE8C09BC452C80CCCCBCF8ED354D71FDBEDDEBFE296E670EA4EEE30F2E8
:2002200016F60001020000001400FFFFFF000102000000140001FFFF560ADB0952091124B4
:200240001FBECFE5D4E0DEBFCDBF14BE88E10FB6F89481BD11BC0FBE10E0A0E6B0E0E6E6FA
:20026000FBE102C005900D92A836B107D9F711E0A8E6B0E001C01D92A43AB107E1F72CD05D
:2002800070CCBECEFC01108211820895DC0111968C91119790E0FD01E80FF91F6283019695
:2002A0008F73907011968C930895DC012C9130E0FC01E20FF31F82812F5F3F4F2F733070CE
:2002C0002C930895FC018181E0818E1710F08E1B0895805C8E1B08951FD16CDAF7DA57DA1D
:2002E00085D4BFD77ED9882359F080911401813041F480E06091150146E151E05ED701C003
:200300008DD7789450D1F2D44ED1AFD74CD131D44AD1E4D9F7CFE82FF0E0E053FF4F8081B8
:2003200093818917B9F0891758F4292F281B9585291718F0980F90830895280F20830895A9
:20034000282F291B9585291718F0891B80830895821B80830895E091870093E0E99FF0013B
:200360001124E859FF4F8083728361838091870090E001966AE070E0CADA809387000895C9
:20038000DC01E091860083E0E89FF0011124E859FF4F80818C938181928112969C938E93BD
:2003A00011978091860090E001966AE070E0AFDA809386000895282F80918700882311F4FF
:2003C00089E001C0815090E0FC01EE0FFF1FE80FF91FE859FF4F208308958F929F92AF9229
:2003E000BF92DF92EF92FF920F931F93CF93DF937C0164E6A62E60E0B62E950180E0782FA5
:200400007F5F472F15C0C42FD0E0CC59DF4F6881F9015081F701E60FF11DD701A50FB11DB4
:2004200090818C91981718F4F901608358834F5F433048F32F5F3F4F872F733001F710E062
:20044000F70180818B3008F011E0F70181818B3008F01260F70182818B3008F01460812F0E
:2004600068EE7DEF78DFDD2451E0852E912CF5018081C82FD0E0F701EC0FFD1F0081802FE4
:200480008B50843F68F5F4EBFD1530F0053B20F0812F68EE7DEF5FDFD016C0F4C4010C2EB7
:2004A00002C0880F991F0A94E2F780951823CE0DDF1D8881E82FF0E0EE0FFF1FEC5DFF4FEB
:2004C00065917491812F47DFD02E0AC0C40102C0880F991FCA95E2F780951823812F6BDF2B
:2004E0000894A11CB11C87E6A81680E0B80609F0BECFE4EBED1520F0812F68EE7DEF2BDFAA
:20050000DF91CF911F910F91FF90EF90DF90BF90AF909F908F900895A3E0B0E0E1E9F2E016
:2005200017CA88B3887F88BB82B38F7182BB87B3876087BB81B3806E81BB89E08EBD89B72E
:20054000886189BF80E09AEF9BBD8ABD88EE9DEF99BD88BD81E08093DA008093DD008093F4
:20056000DB008093DE008093DC008093DF0000ED10E0C80132DFC80130DFCE01019600DFFA
:20058000898180938F0010928E002396E4E0FCC98091870090918600891710F0891B08951D
:2005A000865F891B089503C080ED90E016DFF0DF8530D0F30895A0E0B0E0E0EEF2E0C0C963
:2005C000EC01ED814E81EE2319F44883498388C08B819C8168E671E086D96C016CE370E0C1
:2005E00082D92FEF30E0BC01629FC001639F900D729F900D11244E966CE370E074D97B0125
:20060000F0E0C9018E1B9F0B042F10E0BC01609FC001619F900D709F900D112480589F4F09
:200620006FEF70E074D95B01EE9EC001EF9E900DFE9E900D112480589F4F6FEF70E053D9DE
:20064000C901861B970BBC01609FC001619F900D709F900D112480589F4F6FEF70E043D902
:200660004B01C9018E199F09BC016E9FC0016F9F900D7E9F900D11246FEF70E034D9261BF4
:20068000370B209FC001219F900D309F900D11246FEF70E028D99B01C6016CE370E023D9ED
:2006A0006230A9F0633028F4662351F06130E9F40AC0643099F0643070F06530B1F412C041
:2006C0004883298302C088824983AA820EC0A88249832A830AC0A882898202C02883A982D7
:2006E0004A8303C04883A9828A82CDB7DEB7ECE043C91F93CF93DF93FC019081818152810E
:20070000282F891708F4292F322F251708F4352F36831582332301F1981708F4892F482F1F
:20072000581708F4452F132F141BC12FD0E08FEF90E0BC01C69FC001C79F900DD69F900DE3
:200740001124232F2695632F70E0820F911DDFD86583341729F44EC015821482138252C04D
:20076000512F5695408121813417B1F4822F90E02281821B91092CE330E0BC01629FC00122
:20078000639F900D729F900D1124850F911DBE01BED868597E4F30C082813217A1F490E071
:2007A000841B91092CE330E0BC01629FC001639F900D729F900D1124850F911DBE01A7D860
:2007C00068587F4F19C03817A9F4842F90E0821B91092CE330E0BC01629FC001639F900D2F
:2007E000729F900D1124850F911DBE0190D860517F4F02C060E070E0CB0168E671E073D826
:2008000094838383DF91CF911F910895E3EDF0E0DF01139783E00D9001928150E1F7109296
:200820008E000895681710F4861B0895681B862F08958F929F92BF92CF92DF92EF92FF9270
:200840000F931F93DF93CF930F92CDB7DEB7B82EC62E00ED10E04801DD24FF2490E0F4012D
:20086000838160819983DEDF9981F81610F4D92EF82E9F5F0894811C911C933081F7ED2D28
:20088000F0E0E053FF4FB586C286EE248F2C9924ED14C1F0F80183816081C4DF882359F0D3
:2008A000682F70E086959401280F311DC9012FD8862F662309F481E08C9D802D1124F801AB
:2008C0008287B586E3940F5F1F4FF3E0EF1601F70F90CF91DF911F910F91FF90EF90DF9075
:2008E000CF90BF909F908F9008959091D3008091D000981779F49091D4008091D1009817E8
:2009000049F420E09091D5008091D200981719F421E001C020E0822F0895E3EDF0E0DC0178
:2009200090818C91282F332727FD3095290F311D2F3F310521F01CF02FEF30E004C037FF80
:2009400002C020E030E02193119680E0E63DF80739F7862F642F6DDF10928E0008950F93B5
:200960001F93CF93DF93EC01162F042F83ED90E0C0DE888199812091D6003091D700820F3B
:20098000931F9093D7008093D6009091D8008A81282F332727FD3095290F311D2F3F3105FA
:2009A00021F01CF02FEF30E004C037FF02C020E030E02093D8009091D9008B81282F3327DE
:2009C00027FD3095290F311D2F3F310521F01CF02FEF30E004C037FF02C020E030E020933A
:2009E000D90083ED90E0E7DD812F602F22DF10928E00DF91CF911F910F9108951F920F92FB
:200A00000FB60F9211240F931F932F933F934F935F936F937F938F939F93AF93BF93EF9301
:200A2000FF93DF93CF9300D00F92CDB7DEB790918F0088B3887F892B88BB82B39295990FD9
:200A4000907E8F71982B92BB8E010F5F1F4F11C08CB59DB582179307D8F388B39981887F4F
:200A6000892B88BB82B39295990F907E8F71982B92BBC80185DC8CB59DB52A813B818C5954
:200A80009F4F2817390720F339BD28BD898180938F000F900F900F90CF91DF91FF91EF9192
:200AA000BF91AF919F918F917F916F915F914F913F912F911F910F910F900FBE0F901F90DC
:200AC0001895EF92FF920F931F938C01862FF42E6091E100ACD0E82E8F2D6091E200A7D035
:200AE000682FF80180818093D30081818093D40082818093D500662309F461E08E2D99DEB2
:200B000010928E001F910F91FF90EF900895CF92DF92EF92FF920F931F937C01862F142FFD
:200B20006091E10084D0C82E812F6091E2007FD0D82E06ED10E0F70180819181A281B3817C
:200B40008093D6009093D700A093D800B093D900C80198D0C80103972EDD8C2D6D2D69DE52
:200B600010928E001F910F91FF90EF90DF90CF900895EF92FF920F931F93CF93DF93C0ED95
:200B8000D0E008E810E0FF24F394EE2480918E008F2169F0C8011CD6882349F08E2DBBDB71
:200BA0008F2D809590918E00892380938E0080918E008F2171F498818B81981751F06A85B0
:200BC000662339F0C801FED580918E008F2980938E00E39421960E5F1F4F83E0E81611F064
:200BE000FF0CD4CFCDB7DEB7E6E0CCC6A298AA9AA39AAB988FEF8093E5008093E6008A9847
:200C000092989A9903C081E08093E700089580910001882311F48A9A9298089580910001FD
:200C2000882321F08A989298109200010895482F67FF10C0282F30E0862F992787FD90953A
:200C4000909581959F4F8217930714F041E010C0460F0EC0662361F0772767FD7095680FC8
:200C6000711D6F3F710519F010F04FEF01C0462F842F0895689FC00111246FEF70E033D641
:200C8000CB0108950F931F938C01FC01808191812091E3003091E400820F931F9183808367
:200CA00082816091E500E6DFF801828383816091E600E0DFF80183831F910F910895189565
:200CC00082E691E0FFDA8823D9F75D9BF9CF08951F93CF93DF93EC0110E08991F1D51F5FC9
:200CE0001F30D9F7DF91CF911F910895A8E1B0E0EBE7F6E02EC680E291E0E4DA882389F14D
:200D000080E291E0D2DA182F8091F8008F3089F41093E000812F8F5FD3D51092F70081E005
:200D20008093F9001092FB001092FA001092E7000EC0812FC5D58091F7008F3040F4E82FBB
:200D4000F0E0E851FF4F10838F5F8093F7001B3131F48091F8008F5F8093F80002C01092DA
:200D6000F8008091F900882309F472C18091FA009091FB00009729F08C3B910509F064C144
:200D800006C08CEB90E09093FB008093FA008091F7008F3009F05CC19091E8008091E000A4
:200DA000981719F09F3F09F04CC18091E900873009F4B7C0883088F48330A9F1843030F419
:200DC000813009F1823009F03CC125C0853009F46DC0863008F08CC047C08A3009F4CAC0BA
:200DE0008B3038F4883009F4A5C0893009F029C1A9C08C3009F4FDC08C3008F4D1C0803876
:200E000009F01FC1D8C08CEE90E06091EA004091EB0057DE16C18CEE90E06091EA0040913E
:200E2000EB0075DE0EC12091EA002C3308F009C18091EB0089838091EC008A838091ED00D9
:200E40009091EE009C838B838FEF88878091EF008D838091F0008E838091F1008F83822FE2
:200E6000BE016F5F7F4F42C02091EA002C3308F0E8C08091EB0089878091EC008A87809150
:200E8000ED009091EE009C878B878091EF009091F000988B8F878091F1008D878091F200BE
:200EA0008E87822FBE01675F7F4F20C02091EA002C3308F0C6C08091EB00898B8091EC00B4
:200EC0008A8B8091ED009091EE009C8B8B8B8FEF888F8091D0008D8B8091D1008E8B809119
:200EE000D2008F8B822FBE016F5E7F4FA5D3A9C08091EA008093E1008091EB008093E2003A
:200F00008091EC009091ED009093E4008093E3008091EE008093E5008091EF008093E600D9
:200F200090C041D173DC80E06091EA004BEE50E044D187C038D18091EA00882309F481C013
:200F400065DC7FC080910101882309F47AC0CDDC882309F476C08CEE90E06091EA004091FF
:200F6000EB00DBDC8FEE90E06091EA004091EB00F6DC67C04CDE6091EA00662311F465E07A
:200F800008C0643310F06FEF04C085E0689F602D11248EEF90E016D482E08093000151C044
:200FA000A4E1B1E0EAEEF0E08CE001900D928150E1F7F4D246C08091EA008B3609F041C0AC
:200FC0008091EB00863509F03CC08091EC00873209F037C08091ED008C3F99F571DE2BE00E
:200FE00088E190E00FB6F894A89581BD0FBE21BD28C085B78F78806285BF62DE98B325B3ED
:2010000032B347B354B361B318BA15BA12BA17BA14BA11BA84E082BB80E48ABF8BB780648B
:201020008BBF85B7806885BF889585B78F7785BF8BB78F7B8BBF98BB25BB32BB47BB54BB94
:2010400061BB1092F7009DCE1092FB001092FA0080910001823029F48EEF90E0B9D381114B
:20106000DDDD8091E700882309F49AC08091FC009091FD008C3F9105C1F08D3F910518F411
:20108000892B59F089C021E08231920709F44DC08F51914009F080C064C085E990E064E182
:2010A00091D303C08CEF90E057C085E990E090D38823C1F38FEF8093970087E0809398002D
:2010C00082E292E09093920080939100109290005DC069D09BDBE0919100F0919200319607
:2010E000F0939200E09391003197E491E0939900AAE9B0E0E0919100F09192003196F0930C
:201100009200E09391003197E491ED9380E0A43AB80781F710E08BE1D3D31F5F1F30D9F768
:2011200081E0CED382E191E017C087E990E0D0DD80E0609199004AE950E03FD084E893E03A
:20114000909394008093930011C085E990E064E639D307C08FE191E09093FD008093FC0056
:201160001FC085E990E034D38823A1F3809193009091940001979093940080939300019687
:2011800021F7809190008F5F8093900080919000823008F095CF9DCF1092FD001092FC00AD
:2011A0006896E3E0F2C310920601109205011092040181E0809301010895633070F5109214
:2011C0000101282F30E0F90174E0EE0FFF1F7A95E1F7E21BF30BE95FFE4FDA018AE00D90E4
:2011E00001928150E1F7E62FF0E0EE0FFF1FE85CFD4F85919491F90144E0EE0FFF1F4A95D0
:20120000E1F7E21BF30BEF5FFE4F9283818381E0858381E191E06AE0D5C20895AAE0B0E073
:20122000E3E1F9E097C387E190E09A8389838B818E7F82608B838CE38A878FEF8887898790
:2012400081E08C8383E08D8384E690E09F838E8380E061E0AE014F5F5F4FAFDF2A96E2E0E2
:2012600095C381E191E064E1ADC2809101018823C1F481E191E0ACD2882399F0809106017F
:20128000882359F0E0910201F091030182E091E00995823014F01092060181E191E06AE074
:2012A00091C20895A7E0B0E0E7E5F9E051C38C01FC0182819381009729F0823C910509F0D0
:2012C00073C066C0F80185818093AD001092AC008091AD0064EA70E095D18091AB008F3F5C
:2012E00089F48091A80089838091A9008A838091AA008B83CE0101966091A4004091A500AB
:20130000E0DB13C08091AA009091AB009D838C838091A8008E838091A9008F83CE0104968A
:201320006091A4004091A500F2DB8091AC009091AD008823D1F4F80186819817E1F487814E
:20134000813051F0813018F0823011F50AC0F8011382128282E02CC0F80185818093AD0031
:2013600017C081E08093AC000AC0F8018581981731F41092AC009F5F9093AD0009C0915013
:20138000FBCF82EC90E0F8019383828381E010C08091A6009091A70001979093A70080936C
:2013A000A600019671F794CFF8011382128283E02796E4E0E9C2CF93DF93EC018A819B818C
:2013C0008837910509F44EC08F37910509F45CC0892B09F065C06D817E818F8180FF05C025
:2013E0008091E00090E06827792780E090E027D38D858093B1008C858093B0001DD3DC011C
:20140000CB0168E671E06FD2BC018E85482F50E041155105B9F02091AE003091AF00261B44
:20142000370B37FF03C0309521953F4F253B310534F088E691E0FC01E21BF30B9F012417FC
:201440003507E4F27093AF006093AE008EEA90E0688549855CDB8F8181FF07C088E790E017
:201460009B838A8342DA8823F1F08A859B85009729F29093B3008093B20006C08FE790E071
:201480009B838A8381E00FC08091B2009091B30001979093B3008093B200019679F7AECFA3
:2014A0001B821A8283E0DF91CF910895CF93DF93EC018A819B818434910509F45DC085341A
:2014C000910508F065C0009721F0CF9709F060C040C0488559855093B5004093B4008E8555
:2014E0008093B7008D858093B6002091E00030E08C85992787FD9095B901689F9001699FD2
:20150000300D789F300D11248A859B85BC01269FC001279F900D369F900D1124840F951F42
:201520009093B5008093B40084EB90E06D814E81EEDA8A859B852091B4003091B500820F0D
:20154000931F9093B5008093B4008FE390E09B838A83CBD98823F9F08F812AE0829FC001F9
:2015600011249093B9008093B80006C084E490E09B838A8381E00FC08091B8009091B900F3
:2015800001979093B9008093B800019679F7CCCF1B821A8283E0DF91CF9108958091CE0082
:2015A0008823F1F483E280931301ABEBB0E0E3E1F1E08DE001900D928150E1F71092C800A4
:2015C0008DE08093CB0080E090E09093CA008093C90081E08093CE00109213018093BA0062
:2015E00008958091BA00882319F480E090E0089590E080911301833209F091E081E098278A
:20160000892F08959B01682F70E083E0660F771F8A95E1F7635F7F4FC90148E050E018C201
:201620008091BA00882339F083E191E060E070E04DE050E00DC20895982F8091CE0088238C
:20164000E9F4ABEBB0E0FB0188E001900D928150E1F71092C80088E08093CB00892F90E072
:2016600023E0880F991F2A95E1F7835F9F4F9093CA008093C90081E08093CE0008950F9367
:201680001F93CF93DF93C0E0D0E080E090E08C010F5F1F4FEDD1C8278C2F82958C27082ED3
:2016A000869586958025082E8695802587700C2ECD2F869507948795D02DC82706948795B8
:2016C000D025C82781E00D3E180711F0C801DFCFCE01DF91CF911F910F9108952091CE00D8
:2016E000222309F453C08091CC009091CD0084369105E1F18536910538F4009741F08E35A0
:20170000910509F03FC020C08C369105D9F5213091F57DDA1BC08091C9009091CA000196D0
:201720009093CA008093C90001972091C800E22FF0E0E654FF4F61812F5F2093C800A5D105
:2017400003C08EE590E019C0E199FBCF8091CB0081508093CB008F5FF1F691DFBC018DEEBE
:2017600091E0A0D103C084E690E007C0E199FBCF55DA1092CE008CE690E09093CD0080935B
:20178000CC0008951092CD001092CC0008950F931F9375DF8C018DEE91E072D11092BA00A6
:2017A0000817190719F481E08093BA0039DF1F910F9108958CE983BD8FE085BD89B780681C
:2017C00089BF0895FC018091CF00808361830895FC012181222311F481E008959091CF00EC
:2017E0008081891711F480E00895215021838091CF00808380E0089578941F920F920FB62E
:201800000F9211248F938091CF008F5F8093CF008F910F900FBE0F901F9018951F920F9247
:201820000FB60F9211242F933F934F935F936F937F938F939F93AF93BF93EF93FF9382E62D
:2018400091E033D58CB982E691E03CD5882309F45598FF91EF91BF91AF919F918F917F914B
:201860006F915F914F913F912F910F900FBE0F901F9018951F920F920FB60F9211242F93F2
:201880003F934F935F936F937F938F939F93AF93BF93EF93FF936CB180E291E0F7D4FF9147
:2018A000EF91BF91AF919F918F917F916F915F914F913F912F910F900FBE0F901F901895F1
:2018C000682F82E691E0E2D4559A089510BC83E389B986E880BD88E98AB980E291E0D2D40A
:2018E00082E691E0CFC4AA1BBB1B51E107C0AA1FBB1FA617B70710F0A61BB70B881F991FE8
:201900005A95A9F780959095BC01CD01089597FB092E07260AD077FD04D0E5DF06D0002004
:201920001AF4709561957F4F0895F6F7909581959F4F08952F923F924F925F926F927F920A
:201940008F929F92AF92BF92CF92DF92EF92FF920F931F93CF93DF93CDB7DEB7CA1BDB0BB3
:201960000FB6F894DEBF0FBECDBF09942A88398848885F846E847D848C849B84AA84B984D0
:20198000C884DF80EE80FD800C811B81AA81B981CE0FD11D0FB6F894DEBF0FBECDBFED0123
:2019A0000895A0E0B0E0E6EDFCE0CCCFEC01A880B980CA80DB80A114B104C104D10441F404
:2019C00084E2A82E89EDB82E8BE5C82E87E0D82EC601B5012DE133EF41E050E085D027EA38
:2019E00031E440E050E061D07B018C01C601B5012DE133EF41E050E077D0CA01B9012CEE64
:201A000034EF4FEF5FEF51D06E0D7F1D801F911F97FF04C061507040804090486883798356
:201A20008A839B839B01AC015F77B901CA01CDB7DEB7EAE0A3CFB5CF80E690E0B2CF6093B4
:201A400060007093610080936200909363000895DC01CB01FC01E199FECF06C0FFBBEEBB14
:201A6000E09A31960DB20D9241505040B8F70895E199FECF9FBB8EBBE09A99278DB3089559
:201A8000A8E1B0E042E050E0E5CF262FE199FECF9FBB8EBB2DBB0FB6F894E29AE19A0FBEEB
:201AA00001960895F2DF272FF1CF629FD001739FF001829FE00DF11D649FE00DF11D929FEB
:201AC000F00D839FF00D749FF00D659FF00D9927729FB00DE11DF91F639FB00DE11DF91F60
:201AE000BD01CF011124089597FB092E05260ED057FD04D014D00AD0001C38F450954095CC
:201B0000309521953F4F4F4F5F4F0895F6F790958095709561957F4F8F4F9F4F0895A1E2F7
:201B20001A2EAA1BBB1BFD010DC0AA1FBB1FEE1FFF1FA217B307E407F50720F0A21BB30B44
:201B4000E40BF50B661F771F881F991F1A9469F760957095809590959B01AC01BD01CF0103
:201B60000895F894FFCF0100000000010200FFFFFFFFFFFFFFFFFFFFFFFFFFFFFFFFFFFF7C
:201B8000FFFFFFFFFFFFFFFFFFFFFFFFFFFFFFFFFFFFFFFFFFFFFFFFFFFFFFFFFFFFFFFF65
:201BA000FFFFFFFFFFFFFFFFFFFFFFFFFFFFFFFFFFFFFFFFFFFFFFFFFFFFFFFFFFFFFFFF45
:201BC000FFFFFFFFFFFFFFFFFFFFFFFFFFFFFFFFFFFFFFFFFFFFFFFFFFFFFFFFFFFFFFFF25
:201BE000FFFFFFFFFFFFFFFFFFFFFFFFFFFFFFFFFFFFFFFFFFFFFFFFFFFFFFFFFFFFFFFF05
:201C000000C011241FBECFE5D4E0DEBFCDBF14BE88E10FB6F89481BD11BC0FBE10E0A0E687
:201C2000B0E0E6ECFFE102C005900D92A036B107D9F712E0A0E6B0E001C01D92AC37B107FB
:201C4000E1F732D0BEC1DCCF8627282F22952827022E269526952025022E269520252770C4
:201C6000082E892F269507942795902D8227069427959025822708955D9BFECF8CB9089506
:201C800018BA17BA12BA11BA10BC19B880E48BB91AB81EBC1BBC1ABC1DBC1CBC88B788BF35
:201CA000E0E0F0E0099508958DE093E09BBD8ABD8DE08EBDE0E0F0E0859194918F5F9F4F7B
:201CC00031F0929A8CB58230E8F3829970C110BC83E389B986E880BD88E18AB987E087BB29
:201CE00077247394DD24D394A3E06A2EF5E0BF2EE1E1AE2E72E0972E60E1862E54E0C52E2C
:201D00005F9B27C01CB1809162008F3051F410936300812F8F5FB0DF10926800D09261009E
:201D20000EC0812FA9DF809168008F3040F4E82FF0E0EF59FF4F10878F5F809368001B3168
:201D400031F4809162008F5F8093620002C01092620080916100882309F400C1809168006E
:201D60008F3009F0FBC09091690080916300981719F09F3F09F0F0C080916A00843809F47F
:201D800042C0853840F48238C9F08338E0F4813809F0D8C00AC0863809F478C0863808F48D
:201DA0004EC0873809F0CEC0C9C080916B0090916C0090937B0080937A00C4C01092790073
:201DC00010927800BFC02091780030917900C9010D968150924010F40DE002C0022F01957D
:201DE00010E0C90184589F4F6BE670E0A801E0D08091780090917900080F191F10937900D7
:201E0000009378009FC0C0916B00D0916C000CE710E02FEF3FEF07C0F80161918F01C90194
:201E200013DF9C0121972097B9F780916D0090916E002817390739F180916F001FC000914E
:201E40006B0010916C00C0916D00D0916E002FEF3FEF09C0F8010F5F1F4FE491C9016E2FB7
:201E6000F3DE9C0121972097A9F780916F00909170002817390739F0809171008093650032
:201E8000109264005FC0D09264005CC08A9A00917A0010917B0080917800909179009C0130
:201EA00046E0369527954A95E1F78F739070892B09F02F5FB801ACE7B0E030E086E0220FFE
:201EC000331F8A95E1F77D01E20EF31E2CC0C19AFB0160925700E89507B600FCFDCFED01BE
:201EE00040E050E0FB01E40FF51F899199910C0170925700E895112407B600FCFDCF4E5F01
:201F00005F4F4034510571F7A05CBF4FFB01B0925700E89507B600FCFDCFA0925700E8953A
:201F2000C198605C7F4FAE15BF0589F6020F131F10937B0000937A008A9804C0D09266009C
:201F40009092670080916500882331F080916400882311F48A9AC09A1092680008B604FE49
:201F6000CFCE88BE809160008F5F809360008150843129F488B38C2588BB109260008A9BB3
:201F800009C080916500815080936500882311F48A98C09880916600882309F4B1CE8091E0
:201FA00067008150809367008F5F09F0A9CE68DEFB01DC0102C001900D9241505040D8F710
:061FC0000895F894FFCF24
:00000001FF
